 jabswitch

 Timestamp is ffffffff (Sun Feb  7 06:28:15 2106)

 Preferred load address is 00400000

 Start         Length     Name                   Class
 0001:00000000 0000376bH .text$mn                CODE
 0002:00000000 000001a0H .idata$5                DATA
 0002:000001a0 00000004H .00cfg                  DATA
 0002:000001a4 00000004H .CRT$XCA                DATA
 0002:000001a8 00000004H .CRT$XCAA               DATA
 0002:000001ac 00000004H .CRT$XCZ                DATA
 0002:000001b0 00000004H .CRT$XIA                DATA
 0002:000001b4 00000004H .CRT$XIAA               DATA
 0002:000001b8 00000004H .CRT$XIAC               DATA
 0002:000001bc 00000004H .CRT$XIZ                DATA
 0002:000001c0 00000004H .CRT$XPA                DATA
 0002:000001c4 00000004H .CRT$XPZ                DATA
 0002:000001c8 00000004H .CRT$XTA                DATA
 0002:000001cc 00000004H .CRT$XTZ                DATA
 0002:000001d0 00000000H .gfids$y                DATA
 0002:000001d0 00001100H .rdata                  DATA
 0002:000012d0 00000130H .rdata$r                DATA
 0002:00001400 00000004H .rdata$sxdata           DATA
 0002:00001404 000002d8H .rdata$zzzdbg           DATA
 0002:000016dc 00000004H .rtc$IAA                DATA
 0002:000016e0 00000000H .rtc$IMZ                DATA
 0002:000016e0 00000004H .rtc$IZZ                DATA
 0002:000016e4 00000004H .rtc$TAA                DATA
 0002:000016e8 00000000H .rtc$TMZ                DATA
 0002:000016e8 00000008H .rtc$TZZ                DATA
 0002:000016f0 000000ecH .xdata$x                DATA
 0002:000017dc 00000000H .edata                  DATA
 0002:000017dc 00000104H .idata$2                DATA
 0002:000018e0 00000014H .idata$3                DATA
 0002:000018f4 000001a0H .idata$4                DATA
 0002:00001a94 00000792H .idata$6                DATA
 0003:00000000 00000048H .data                   DATA
 0003:00000048 00000078H .data$r                 DATA
 0003:000000c0 0000038cH .bss                    DATA
 0004:00000000 00000120H .rsrc$01                DATA
 0004:00000120 00000600H .rsrc$02                DATA

  Address         Publics by Value              Rva+Base       Lib:Object

 0000:00000000       ___guard_fids_count        00000000     <absolute>
 0000:00000000       ___guard_iat_table         00000000     <absolute>
 0000:00000000       ___guard_iat_count         00000000     <absolute>
 0000:00000000       ___dynamic_value_reloc_table 00000000     <absolute>
 0000:00000000       ___hybrid_code_map         00000000     <absolute>
 0000:00000000       ___guard_fids_table        00000000     <absolute>
 0000:00000000       ___guard_longjmp_count     00000000     <absolute>
 0000:00000000       ___enclave_config          00000000     <absolute>
 0000:00000000       ___volatile_metadata       00000000     <absolute>
 0000:00000000       ___guard_longjmp_table     00000000     <absolute>
 0000:00000000       ___hybrid_auxiliary_iat    00000000     <absolute>
 0000:00000000       ___hybrid_code_map_count   00000000     <absolute>
 0000:00000001       ___safe_se_handler_count   00000001     <absolute>
 0000:00000100       ___guard_flags             00000100     <absolute>
 0000:00000000       ___ImageBase               00400000     <linker-defined>
 0001:00000010       ?isXP@@YA_NXZ              00401010 f   jabswitch.obj
 0001:000000d0       ?enableJAB@@YAXXZ          004010d0 f   jabswitch.obj
 0001:000005b0       ?disableJAB@@YAXXZ         004015b0 f   jabswitch.obj
 0001:00000860       ?modify@@YAH_N@Z           00401860 f   jabswitch.obj
 0001:00000dd0       ?printUsage@@YAXXZ         00401dd0 f   jabswitch.obj
 0001:00000eb0       ?printVersion@@YAXXZ       00401eb0 f   jabswitch.obj
 0001:00001140       ?regEnable@@YAHXZ          00402140 f   jabswitch.obj
 0001:00001410       ?regDeleteValue@@YAHPAUHKEY__@@PB_W@Z 00402410 f   jabswitch.obj
 0001:00001860       ?regDisable@@YAHXZ         00402860 f   jabswitch.obj
 0001:00001980       _main                      00402980 f   jabswitch.obj
 0001:00001c30       ??$sprintf_s@$0GE@@@YAHAAY0GE@DPBDZZ 00402c30 f i jabswitch.obj
 0001:00001c70       ??$strcat_s@$0BAE@@@YAHAAY0BAE@DPBD@Z 00402c70 f i jabswitch.obj
 0001:00001ca0       ??$strcat_s@$0CAA@@@YAHAAY0CAA@DPBD@Z 00402ca0 f i jabswitch.obj
 0001:00001cd0       ??$strcat_s@$0GE@@@YAHAAY0GE@DPBD@Z 00402cd0 f i jabswitch.obj
 0001:00001d00       ??$strcpy_s@$0CAA@@@YAHAAY0CAA@DPBD@Z 00402d00 f i jabswitch.obj
 0001:00001d30       ??$strcpy_s@$0GE@@@YAHAAY0GE@DPBD@Z 00402d30 f i jabswitch.obj
 0001:00001d60       ?strstr@@YAPADQADQBD@Z     00402d60 f i jabswitch.obj
 0001:00001d80       ?wcsstr@@YAPA_WPA_WPB_W@Z  00402d80 f i jabswitch.obj
 0001:00001da0       ___local_stdio_printf_options 00402da0 f i jabswitch.obj
 0001:00001db0       __vfprintf_l               00402db0 f i jabswitch.obj
 0001:00001df0       __vsprintf_s_l             00402df0 f i jabswitch.obj
 0001:00001e70       _fprintf                   00402e70 f i jabswitch.obj
 0001:00001ed0       _printf                    00402ed0 f i jabswitch.obj
 0001:00001f40       _vsprintf_s                00402f40 f i jabswitch.obj
 0001:00001f66       _GetFileVersionInfoSizeW@8 00402f66 f   version:VERSION.dll
 0001:00001f6c       _GetFileVersionInfoW@16    00402f6c f   version:VERSION.dll
 0001:00001f72       _VerQueryValueW@16         00402f72 f   version:VERSION.dll
 0001:00001f78       ??_U@YAPAXI@Z              00402f78 f   MSVCRT:new_array.obj
 0001:00001f81       ___raise_securityfailure   00402f81 f   MSVCRT:gs_report.obj
 0001:00001fac       ___report_gsfailure        00402fac f   MSVCRT:gs_report.obj
 0001:000020a5       ___report_rangecheckfailure 004030a5 f   MSVCRT:gs_report.obj
 0001:000020b1       ___report_securityfailure  004030b1 f   MSVCRT:gs_report.obj
 0001:0000217f       @_RTC_CheckStackVars@8     0040317f f   MSVCRT:stack.obj
 0001:000021d3       __RTC_CheckEsp             004031d3 f   MSVCRT:stack.obj
 0001:00002202       @__security_check_cookie@4 00403202 f   MSVCRT:secchk.obj
 0001:0000245a       _mainCRTStartup            0040345a f   MSVCRT:exe_main.obj
 0001:00002464       ??2@YAPAXI@Z               00403464 f   MSVCRT:new_scalar.obj
 0001:00002494       ?_RTC_Failure@@YAXPAXH@Z   00403494 f   MSVCRT:error.obj
 0001:000024d0       ?_RTC_StackFailure@@YAXPAXPBD@Z 004034d0 f   MSVCRT:error.obj
 0001:0000282e       ?_RTC_GetErrorFunc@@YAP6AHHPBDH00ZZPBX@Z 0040382e f   MSVCRT:userapi.obj
 0001:00002834       ?_RTC_GetErrorFuncW@@YAP6AHHPB_WH00ZZPBX@Z 00403834 f   MSVCRT:userapi.obj
 0001:0000287e       ___scrt_acquire_startup_lock 0040387e f   MSVCRT:utility.obj
 0001:000028b0       ___scrt_initialize_crt     004038b0 f   MSVCRT:utility.obj
 0001:000028e9       ___scrt_initialize_onexit_tables 004038e9 f   MSVCRT:utility.obj
 0001:0000298e       ___scrt_is_nonwritable_in_current_image 0040398e f   MSVCRT:utility.obj
 0001:00002a22       ___scrt_release_startup_lock 00403a22 f   MSVCRT:utility.obj
 0001:00002a3f       ___scrt_uninitialize_crt   00403a3f f   MSVCRT:utility.obj
 0001:00002a67       __onexit                   00403a67 f   MSVCRT:utility.obj
 0001:00002aa2       _atexit                    00403aa2 f   MSVCRT:utility.obj
 0001:00002b04       ___security_init_cookie    00403b04 f   MSVCRT:gs_support.obj
 0001:00002b4f       __get_startup_new_mode     00403b4f f   MSVCRT:new_mode.obj
 0001:00002b4f       ___scrt_stub_for_initialize_mta 00403b4f f   MSVCRT:utility_desktop.obj
 0001:00002b4f       ___scrt_initialize_winrt   00403b4f f   MSVCRT:utility_desktop.obj
 0001:00002b4f       __matherr                  00403b4f f   MSVCRT:matherr.obj
 0001:00002b4f       __get_startup_thread_locale_mode 00403b4f f   MSVCRT:thread_locale.obj
 0001:00002b4f       __get_startup_commit_mode  00403b4f f   MSVCRT:commit_mode.obj
 0001:00002b4f       ___scrt_exe_initialize_mta 00403b4f f   MSVCRT:utility_desktop.obj
 0001:00002b52       __get_startup_argv_mode    00403b52 f   MSVCRT:argv_mode.obj
 0001:00002b56       __get_startup_file_mode    00403b56 f   MSVCRT:file_mode.obj
 0001:00002b5c       ?__scrt_initialize_type_info@@YAXXZ 00403b5c f   MSVCRT:tncleanup.obj
 0001:00002b68       ___scrt_stub_for_acrt_uninitialize 00403b68 f   MSVCRT:ucrt_stubs.obj
 0001:00002b68       ___acrt_initialize         00403b68 f   MSVCRT:ucrt_stubs.obj
 0001:00002b68       ___acrt_uninitialize       00403b68 f   MSVCRT:ucrt_stubs.obj
 0001:00002b68       ___vcrt_initialize         00403b68 f   MSVCRT:ucrt_stubs.obj
 0001:00002b68       __should_initialize_environment 00403b68 f   MSVCRT:env_mode.obj
 0001:00002b68       ___vcrt_uninitialize       00403b68 f   MSVCRT:ucrt_stubs.obj
 0001:00002b68       ___scrt_stub_for_acrt_initialize 00403b68 f   MSVCRT:ucrt_stubs.obj
 0001:00002b6b       __initialize_default_precision 00403b6b f   MSVCRT:default_precision.obj
 0001:00002b8c       __initialize_denormal_control 00403b8c f   MSVCRT:denormal_control.obj
 0001:00002b8c       @_guard_check_icall_nop@4  00403b8c f   MSVCRT:guard_support.obj
 0001:00002b8c       __initialize_invalid_parameter_handler 00403b8c f   MSVCRT:invalid_parameter_handler.obj
 0001:00002b8d       ___local_stdio_scanf_options 00403b8d f i MSVCRT:default_local_stdio_options.obj
 0001:00002b93       ___scrt_initialize_default_local_stdio_options 00403b93 f   MSVCRT:default_local_stdio_options.obj
 0001:00002bb0       ___scrt_is_user_matherr_present 00403bb0 f   MSVCRT:matherr_detection.obj
 0001:00002bbc       ___scrt_get_dyn_tls_init_callback 00403bbc f   MSVCRT:dyn_tls_init.obj
 0001:00002bc2       ___scrt_get_dyn_tls_dtor_callback 00403bc2 f   MSVCRT:dyn_tls_dtor.obj
 0001:00002bc8       ___scrt_fastfail           00403bc8 f   MSVCRT:utility_desktop.obj
 0001:00002ce2       ___scrt_initialize_mta     00403ce2 f   MSVCRT:utility_desktop.obj
 0001:00002ce7       ___scrt_is_managed_app     00403ce7 f   MSVCRT:utility_desktop.obj
 0001:00002d2a       ___scrt_set_unhandled_exception_filter 00403d2a f   MSVCRT:utility_desktop.obj
 0001:00002d36       ___scrt_unhandled_exception_filter@4 00403d36 f   MSVCRT:utility_desktop.obj
 0001:00002d77       __crt_debugger_hook        00403d77 f   MSVCRT:utility_desktop.obj
 0001:00002d7f       __RTC_Initialize           00403d7f f   MSVCRT:initsect.obj
 0001:00002dab       __RTC_Terminate            00403dab f   MSVCRT:initsect.obj
 0001:00002de0       __SEH_prolog4              00403de0 f   MSVCRT:sehprolg4.obj
 0001:00002e26       __SEH_epilog4              00403e26 f   MSVCRT:sehprolg4.obj
 0001:00002e3b       __except_handler4          00403e3b f   MSVCRT:chandler4gs.obj
 0001:00002e5e       ??0bad_alloc@std@@QAE@ABV01@@Z 00403e5e f i MSVCRT:throw_bad_alloc.obj
 0001:00002e79       ??0bad_alloc@std@@QAE@XZ   00403e79 f i MSVCRT:throw_bad_alloc.obj
 0001:00002e91       ??0bad_array_new_length@std@@QAE@ABV01@@Z 00403e91 f i MSVCRT:throw_bad_alloc.obj
 0001:00002eac       ??0bad_array_new_length@std@@QAE@XZ 00403eac f i MSVCRT:throw_bad_alloc.obj
 0001:00002ec4       ??0exception@std@@QAE@ABV01@@Z 00403ec4 f i MSVCRT:throw_bad_alloc.obj
 0001:00002ef0       ??1bad_array_new_length@std@@UAE@XZ 00403ef0 f i MSVCRT:throw_bad_alloc.obj
 0001:00002ef0       ??1bad_alloc@std@@UAE@XZ   00403ef0 f i MSVCRT:throw_bad_alloc.obj
 0001:00002f01       ??_Ebad_alloc@std@@UAEPAXI@Z 00403f01 f i MSVCRT:throw_bad_alloc.obj
 0001:00002f01       ??_Gbad_array_new_length@std@@UAEPAXI@Z 00403f01 f i MSVCRT:throw_bad_alloc.obj
 0001:00002f01       ??_Ebad_array_new_length@std@@UAEPAXI@Z 00403f01 f i MSVCRT:throw_bad_alloc.obj
 0001:00002f01       ??_Eexception@std@@UAEPAXI@Z 00403f01 f i MSVCRT:throw_bad_alloc.obj
 0001:00002f01       ??_Gbad_alloc@std@@UAEPAXI@Z 00403f01 f i MSVCRT:throw_bad_alloc.obj
 0001:00002f01       ??_Gexception@std@@UAEPAXI@Z 00403f01 f i MSVCRT:throw_bad_alloc.obj
 0001:00002f2e       ?__scrt_throw_std_bad_alloc@@YAXXZ 00403f2e f   MSVCRT:throw_bad_alloc.obj
 0001:00002f4b       ?__scrt_throw_std_bad_array_new_length@@YAXXZ 00403f4b f   MSVCRT:throw_bad_alloc.obj
 0001:00002f68       ?what@exception@std@@UBEPBDXZ 00403f68 f i MSVCRT:throw_bad_alloc.obj
 0001:00003163       ?_RTC_GetSrcLine@@YAHPAEPA_WKPAH1K@Z 00404163 f   MSVCRT:pdblkup.obj
 0001:000034a8       ___isa_available_init      004044a8 f   MSVCRT:cpu_disp.obj
 0001:0000363f       ___scrt_is_ucrt_dll_in_use 0040463f f   MSVCRT:ucrt_detection.obj
 0001:0000364b       ??3@YAXPAXI@Z              0040464b f   MSVCRT:delete_scalar_size.obj
 0001:00003659       ??_Gtype_info@@UAEPAXI@Z   00404659 f i MSVCRT:std_type_info_static.obj
 0001:00003659       ??_Etype_info@@UAEPAXI@Z   00404659 f i MSVCRT:std_type_info_static.obj
 0001:0000367c       ??3@YAXPAX@Z               0040467c f   MSVCRT:delete_scalar.obj
 0001:00003681       _IsProcessorFeaturePresent@4 00404681 f   kernel32:KERNEL32.dll
 0001:00003687       _memset                    00404687 f   vcruntime:VCRUNTIME140.dll
 0001:0000368d       _strstr                    0040468d f   vcruntime:VCRUNTIME140.dll
 0001:00003693       _wcsstr                    00404693 f   vcruntime:VCRUNTIME140.dll
 0001:00003699       __except_handler4_common   00404699 f   vcruntime:VCRUNTIME140.dll
 0001:0000369f       ___std_exception_copy      0040469f f   vcruntime:VCRUNTIME140.dll
 0001:000036a5       ___std_exception_destroy   004046a5 f   vcruntime:VCRUNTIME140.dll
 0001:000036ab       __CxxThrowException@8      004046ab f   vcruntime:VCRUNTIME140.dll
 0001:000036b1       ___vcrt_GetModuleFileNameW 004046b1 f   vcruntime:VCRUNTIME140.dll
 0001:000036b7       ___vcrt_LoadLibraryExW     004046b7 f   vcruntime:VCRUNTIME140.dll
 0001:000036bd       _strcpy_s                  004046bd f   ucrt:api-ms-win-crt-string-l1-1-0.dll
 0001:000036c3       _strcat_s                  004046c3 f   ucrt:api-ms-win-crt-string-l1-1-0.dll
 0001:000036c9       _free                      004046c9 f   ucrt:api-ms-win-crt-heap-l1-1-0.dll
 0001:000036cf       _exit                      004046cf f   ucrt:api-ms-win-crt-runtime-l1-1-0.dll
 0001:000036d5       __seh_filter_exe           004046d5 f   ucrt:api-ms-win-crt-runtime-l1-1-0.dll
 0001:000036db       __set_app_type             004046db f   ucrt:api-ms-win-crt-runtime-l1-1-0.dll
 0001:000036e1       ___setusermatherr          004046e1 f   ucrt:api-ms-win-crt-math-l1-1-0.dll
 0001:000036e7       __configure_narrow_argv    004046e7 f   ucrt:api-ms-win-crt-runtime-l1-1-0.dll
 0001:000036ed       __initialize_narrow_environment 004046ed f   ucrt:api-ms-win-crt-runtime-l1-1-0.dll
 0001:000036f3       __get_initial_narrow_environment 004046f3 f   ucrt:api-ms-win-crt-runtime-l1-1-0.dll
 0001:000036f9       __initterm                 004046f9 f   ucrt:api-ms-win-crt-runtime-l1-1-0.dll
 0001:000036ff       __initterm_e               004046ff f   ucrt:api-ms-win-crt-runtime-l1-1-0.dll
 0001:00003705       __exit                     00404705 f   ucrt:api-ms-win-crt-runtime-l1-1-0.dll
 0001:0000370b       __set_fmode                0040470b f   ucrt:api-ms-win-crt-stdio-l1-1-0.dll
 0001:00003711       ___p___argc                00404711 f   ucrt:api-ms-win-crt-runtime-l1-1-0.dll
 0001:00003717       ___p___argv                00404717 f   ucrt:api-ms-win-crt-runtime-l1-1-0.dll
 0001:0000371d       __cexit                    0040471d f   ucrt:api-ms-win-crt-runtime-l1-1-0.dll
 0001:00003723       __c_exit                   00404723 f   ucrt:api-ms-win-crt-runtime-l1-1-0.dll
 0001:00003729       __register_thread_local_exe_atexit_callback 00404729 f   ucrt:api-ms-win-crt-runtime-l1-1-0.dll
 0001:0000372f       __configthreadlocale       0040472f f   ucrt:api-ms-win-crt-locale-l1-1-0.dll
 0001:00003735       __set_new_mode             00404735 f   ucrt:api-ms-win-crt-heap-l1-1-0.dll
 0001:0000373b       ___p__commode              0040473b f   ucrt:api-ms-win-crt-stdio-l1-1-0.dll
 0001:00003741       __callnewh                 00404741 f   ucrt:api-ms-win-crt-heap-l1-1-0.dll
 0001:00003747       _malloc                    00404747 f   ucrt:api-ms-win-crt-heap-l1-1-0.dll
 0001:0000374d       __initialize_onexit_table  0040474d f   ucrt:api-ms-win-crt-runtime-l1-1-0.dll
 0001:00003753       __register_onexit_function 00404753 f   ucrt:api-ms-win-crt-runtime-l1-1-0.dll
 0001:00003759       __crt_atexit               00404759 f   ucrt:api-ms-win-crt-runtime-l1-1-0.dll
 0001:0000375f       __controlfp_s              0040475f f   ucrt:api-ms-win-crt-runtime-l1-1-0.dll
 0001:00003765       _terminate                 00404765 f   ucrt:api-ms-win-crt-runtime-l1-1-0.dll
 0002:00000000       __imp__RegOpenKeyExW@20    00405000     advapi32:ADVAPI32.dll
 0002:00000004       __imp__RegQueryValueExW@24 00405004     advapi32:ADVAPI32.dll
 0002:00000008       __imp__RegSetValueExW@24   00405008     advapi32:ADVAPI32.dll
 0002:0000000c       __imp__RegCloseKey@4       0040500c     advapi32:ADVAPI32.dll
 0002:00000010       \177ADVAPI32_NULL_THUNK_DATA 00405010     advapi32:ADVAPI32.dll
 0002:00000014       __imp__GetProcAddress@8    00405014     kernel32:KERNEL32.dll
 0002:00000018       __imp__FreeLibrary@4       00405018     kernel32:KERNEL32.dll
 0002:0000001c       __imp__VirtualQuery@12     0040501c     kernel32:KERNEL32.dll
 0002:00000020       __imp__GetProcessHeap@0    00405020     kernel32:KERNEL32.dll
 0002:00000024       __imp__HeapFree@12         00405024     kernel32:KERNEL32.dll
 0002:00000028       __imp__HeapAlloc@12        00405028     kernel32:KERNEL32.dll
 0002:0000002c       __imp__GetCurrentProcessId@0 0040502c     kernel32:KERNEL32.dll
 0002:00000030       __imp__ProcessIdToSessionId@8 00405030     kernel32:KERNEL32.dll
 0002:00000034       __imp__GetVersionExW@4     00405034     kernel32:KERNEL32.dll
 0002:00000038       __imp__GetModuleFileNameW@12 00405038     kernel32:KERNEL32.dll
 0002:0000003c       __imp__UnhandledExceptionFilter@4 0040503c     kernel32:KERNEL32.dll
 0002:00000040       __imp__SetUnhandledExceptionFilter@4 00405040     kernel32:KERNEL32.dll
 0002:00000044       __imp__GetCurrentProcess@0 00405044     kernel32:KERNEL32.dll
 0002:00000048       __imp__TerminateProcess@8  00405048     kernel32:KERNEL32.dll
 0002:0000004c       __imp__IsProcessorFeaturePresent@4 0040504c     kernel32:KERNEL32.dll
 0002:00000050       __imp__IsDebuggerPresent@0 00405050     kernel32:KERNEL32.dll
 0002:00000054       __imp__RaiseException@16   00405054     kernel32:KERNEL32.dll
 0002:00000058       __imp__MultiByteToWideChar@24 00405058     kernel32:KERNEL32.dll
 0002:0000005c       __imp__WideCharToMultiByte@32 0040505c     kernel32:KERNEL32.dll
 0002:00000060       __imp__QueryPerformanceCounter@4 00405060     kernel32:KERNEL32.dll
 0002:00000064       __imp__GetCurrentThreadId@0 00405064     kernel32:KERNEL32.dll
 0002:00000068       __imp__GetSystemTimeAsFileTime@4 00405068     kernel32:KERNEL32.dll
 0002:0000006c       __imp__InitializeSListHead@4 0040506c     kernel32:KERNEL32.dll
 0002:00000070       __imp__GetModuleHandleW@4  00405070     kernel32:KERNEL32.dll
 0002:00000074       __imp__GetLastError@0      00405074     kernel32:KERNEL32.dll
 0002:00000078       \177KERNEL32_NULL_THUNK_DATA 00405078     kernel32:KERNEL32.dll
 0002:0000007c       __imp__wsprintfW           0040507c     user32:USER32.dll
 0002:00000080       \177USER32_NULL_THUNK_DATA 00405080     user32:USER32.dll
 0002:00000084       __imp___CxxThrowException@8 00405084     vcruntime:VCRUNTIME140.dll
 0002:00000088       __imp____std_exception_destroy 00405088     vcruntime:VCRUNTIME140.dll
 0002:0000008c       __imp____vcrt_GetModuleFileNameW 0040508c     vcruntime:VCRUNTIME140.dll
 0002:00000090       __imp____vcrt_LoadLibraryExW 00405090     vcruntime:VCRUNTIME140.dll
 0002:00000094       __imp__memset              00405094     vcruntime:VCRUNTIME140.dll
 0002:00000098       __imp__strstr              00405098     vcruntime:VCRUNTIME140.dll
 0002:0000009c       __imp__wcsstr              0040509c     vcruntime:VCRUNTIME140.dll
 0002:000000a0       __imp___except_handler4_common 004050a0     vcruntime:VCRUNTIME140.dll
 0002:000000a4       __imp____std_exception_copy 004050a4     vcruntime:VCRUNTIME140.dll
 0002:000000a8       \177VCRUNTIME140_NULL_THUNK_DATA 004050a8     vcruntime:VCRUNTIME140.dll
 0002:000000ac       __imp__VerQueryValueW@16   004050ac     version:VERSION.dll
 0002:000000b0       __imp__GetFileVersionInfoW@16 004050b0     version:VERSION.dll
 0002:000000b4       __imp__GetFileVersionInfoSizeW@8 004050b4     version:VERSION.dll
 0002:000000b8       \177VERSION_NULL_THUNK_DATA 004050b8     version:VERSION.dll
 0002:000000bc       __imp___dupenv_s           004050bc     ucrt:api-ms-win-crt-environment-l1-1-0.dll
 0002:000000c0       \177api-ms-win-crt-environment-l1-1-0_NULL_THUNK_DATA 004050c0     ucrt:api-ms-win-crt-environment-l1-1-0.dll
 0002:000000c4       __imp__remove              004050c4     ucrt:api-ms-win-crt-filesystem-l1-1-0.dll
 0002:000000c8       __imp__rename              004050c8     ucrt:api-ms-win-crt-filesystem-l1-1-0.dll
 0002:000000cc       \177api-ms-win-crt-filesystem-l1-1-0_NULL_THUNK_DATA 004050cc     ucrt:api-ms-win-crt-filesystem-l1-1-0.dll
 0002:000000d0       __imp___set_new_mode       004050d0     ucrt:api-ms-win-crt-heap-l1-1-0.dll
 0002:000000d4       __imp___callnewh           004050d4     ucrt:api-ms-win-crt-heap-l1-1-0.dll
 0002:000000d8       __imp__malloc              004050d8     ucrt:api-ms-win-crt-heap-l1-1-0.dll
 0002:000000dc       __imp__free                004050dc     ucrt:api-ms-win-crt-heap-l1-1-0.dll
 0002:000000e0       \177api-ms-win-crt-heap-l1-1-0_NULL_THUNK_DATA 004050e0     ucrt:api-ms-win-crt-heap-l1-1-0.dll
 0002:000000e4       __imp___configthreadlocale 004050e4     ucrt:api-ms-win-crt-locale-l1-1-0.dll
 0002:000000e8       \177api-ms-win-crt-locale-l1-1-0_NULL_THUNK_DATA 004050e8     ucrt:api-ms-win-crt-locale-l1-1-0.dll
 0002:000000ec       __imp____setusermatherr    004050ec     ucrt:api-ms-win-crt-math-l1-1-0.dll
 0002:000000f0       \177api-ms-win-crt-math-l1-1-0_NULL_THUNK_DATA 004050f0     ucrt:api-ms-win-crt-math-l1-1-0.dll
 0002:000000f4       __imp___register_onexit_function 004050f4     ucrt:api-ms-win-crt-runtime-l1-1-0.dll
 0002:000000f8       __imp___initialize_onexit_table 004050f8     ucrt:api-ms-win-crt-runtime-l1-1-0.dll
 0002:000000fc       __imp__terminate           004050fc     ucrt:api-ms-win-crt-runtime-l1-1-0.dll
 0002:00000100       __imp___controlfp_s        00405100     ucrt:api-ms-win-crt-runtime-l1-1-0.dll
 0002:00000104       __imp___errno              00405104     ucrt:api-ms-win-crt-runtime-l1-1-0.dll
 0002:00000108       __imp__exit                00405108     ucrt:api-ms-win-crt-runtime-l1-1-0.dll
 0002:0000010c       __imp__perror              0040510c     ucrt:api-ms-win-crt-runtime-l1-1-0.dll
 0002:00000110       __imp___seh_filter_exe     00405110     ucrt:api-ms-win-crt-runtime-l1-1-0.dll
 0002:00000114       __imp___set_app_type       00405114     ucrt:api-ms-win-crt-runtime-l1-1-0.dll
 0002:00000118       __imp___cexit              00405118     ucrt:api-ms-win-crt-runtime-l1-1-0.dll
 0002:0000011c       __imp___configure_narrow_argv 0040511c     ucrt:api-ms-win-crt-runtime-l1-1-0.dll
 0002:00000120       __imp___initialize_narrow_environment 00405120     ucrt:api-ms-win-crt-runtime-l1-1-0.dll
 0002:00000124       __imp___get_initial_narrow_environment 00405124     ucrt:api-ms-win-crt-runtime-l1-1-0.dll
 0002:00000128       __imp___initterm           00405128     ucrt:api-ms-win-crt-runtime-l1-1-0.dll
 0002:0000012c       __imp___initterm_e         0040512c     ucrt:api-ms-win-crt-runtime-l1-1-0.dll
 0002:00000130       __imp___exit               00405130     ucrt:api-ms-win-crt-runtime-l1-1-0.dll
 0002:00000134       __imp___register_thread_local_exe_atexit_callback 00405134     ucrt:api-ms-win-crt-runtime-l1-1-0.dll
 0002:00000138       __imp____p___argc          00405138     ucrt:api-ms-win-crt-runtime-l1-1-0.dll
 0002:0000013c       __imp____p___argv          0040513c     ucrt:api-ms-win-crt-runtime-l1-1-0.dll
 0002:00000140       __imp___c_exit             00405140     ucrt:api-ms-win-crt-runtime-l1-1-0.dll
 0002:00000144       __imp___crt_atexit         00405144     ucrt:api-ms-win-crt-runtime-l1-1-0.dll
 0002:00000148       \177api-ms-win-crt-runtime-l1-1-0_NULL_THUNK_DATA 00405148     ucrt:api-ms-win-crt-runtime-l1-1-0.dll
 0002:0000014c       __imp____stdio_common_vsprintf_s 0040514c     ucrt:api-ms-win-crt-stdio-l1-1-0.dll
 0002:00000150       __imp____p__commode        00405150     ucrt:api-ms-win-crt-stdio-l1-1-0.dll
 0002:00000154       __imp__fgets               00405154     ucrt:api-ms-win-crt-stdio-l1-1-0.dll
 0002:00000158       __imp__feof                00405158     ucrt:api-ms-win-crt-stdio-l1-1-0.dll
 0002:0000015c       __imp____stdio_common_vfprintf 0040515c     ucrt:api-ms-win-crt-stdio-l1-1-0.dll
 0002:00000160       __imp___set_fmode          00405160     ucrt:api-ms-win-crt-stdio-l1-1-0.dll
 0002:00000164       __imp__fclose              00405164     ucrt:api-ms-win-crt-stdio-l1-1-0.dll
 0002:00000168       __imp__fopen_s             00405168     ucrt:api-ms-win-crt-stdio-l1-1-0.dll
 0002:0000016c       __imp____acrt_iob_func     0040516c     ucrt:api-ms-win-crt-stdio-l1-1-0.dll
 0002:00000170       __imp__fputs               00405170     ucrt:api-ms-win-crt-stdio-l1-1-0.dll
 0002:00000174       \177api-ms-win-crt-stdio-l1-1-0_NULL_THUNK_DATA 00405174     ucrt:api-ms-win-crt-stdio-l1-1-0.dll
 0002:00000178       __imp__strcat_s            00405178     ucrt:api-ms-win-crt-string-l1-1-0.dll
 0002:0000017c       __imp__strtok_s            0040517c     ucrt:api-ms-win-crt-string-l1-1-0.dll
 0002:00000180       __imp___stricmp            00405180     ucrt:api-ms-win-crt-string-l1-1-0.dll
 0002:00000184       __imp__strcpy_s            00405184     ucrt:api-ms-win-crt-string-l1-1-0.dll
 0002:00000188       __imp___wcslwr_s           00405188     ucrt:api-ms-win-crt-string-l1-1-0.dll
 0002:0000018c       __imp__wcscpy_s            0040518c     ucrt:api-ms-win-crt-string-l1-1-0.dll
 0002:00000190       __imp__wcslen              00405190     ucrt:api-ms-win-crt-string-l1-1-0.dll
 0002:00000194       __imp__wcstok_s            00405194     ucrt:api-ms-win-crt-string-l1-1-0.dll
 0002:00000198       __imp__wcscat_s            00405198     ucrt:api-ms-win-crt-string-l1-1-0.dll
 0002:0000019c       \177api-ms-win-crt-string-l1-1-0_NULL_THUNK_DATA 0040519c     ucrt:api-ms-win-crt-string-l1-1-0.dll
 0002:000001a0       ___guard_check_icall_fptr  004051a0     MSVCRT:guard_support.obj
 0002:000001a4       ___xc_a                    004051a4     MSVCRT:initializers.obj
 0002:000001ac       ___xc_z                    004051ac     MSVCRT:initializers.obj
 0002:000001b0       ___xi_a                    004051b0     MSVCRT:initializers.obj
 0002:000001bc       ___xi_z                    004051bc     MSVCRT:initializers.obj
 0002:000001c0       ___xp_a                    004051c0     MSVCRT:initializers.obj
 0002:000001c4       ___xp_z                    004051c4     MSVCRT:initializers.obj
 0002:000001c8       ___xt_a                    004051c8     MSVCRT:initializers.obj
 0002:000001cc       ___xt_z                    004051cc     MSVCRT:initializers.obj
 0002:00000b68       ??_C@_0NN@NGPKDKPD@The?5value?5of?5ESP?5was?5not?5proper@ 00405b68     MSVCRT:error.obj
 0002:00000c48       ??_C@_0BBN@GPMLNJCF@A?5cast?5to?5a?5smaller?5data?5type?5h@ 00405c48     MSVCRT:error.obj
 0002:00000d68       ??_C@_0BN@FFOINMNJ@Stack?5memory?5was?5corrupted?6?$AN@ 00405d68     MSVCRT:error.obj
 0002:00000d88       ??_C@_0DG@HKJMLLLP@A?5local?5variable?5was?5used?5befor@ 00405d88     MSVCRT:error.obj
 0002:00000dc0       ??_C@_0CM@NGINOKPC@Stack?5memory?5around?5_alloca?5was@ 00405dc0     MSVCRT:error.obj
 0002:00000dec       ??_C@_0BO@GNIAFIKK@Unknown?5Runtime?5Check?5Error?6?$AN@ 00405dec     MSVCRT:error.obj
 0002:00000e10       ??_C@_1GM@OLMCBDMB@?$AAR?$AAu?$AAn?$AAt?$AAi?$AAm?$AAe?$AA?5?$AAC?$AAh?$AAe?$AAc?$AAk?$AA?5?$AAE@ 00405e10     MSVCRT:error.obj
 0002:00000e80       ??_C@_1EA@NFKNIFJP@?$AAR?$AAu?$AAn?$AA?9?$AAT?$AAi?$AAm?$AAe?$AA?5?$AAC?$AAh?$AAe?$AAc?$AAk?$AA?5@ 00405e80     MSVCRT:error.obj
 0002:00000ec0       ??_C@_0BB@PFFGGCJP@Unknown?5Filename@ 00405ec0     MSVCRT:error.obj
 0002:00000ed4       ??_C@_0BE@GNBOBNCK@Unknown?5Module?5Name@ 00405ed4     MSVCRT:error.obj
 0002:00000ee8       ??_C@_0CA@IODNCDPG@Run?9Time?5Check?5Failure?5?$CD?$CFd?5?9?5?$CFs@ 00405ee8     MSVCRT:error.obj
 0002:00000f08       ??_C@_0CG@IAFNJNEE@Stack?5corrupted?5near?5unknown?5va@ 00405f08     MSVCRT:error.obj
 0002:00000f44       ??_C@_0BJ@HEGAHDFO@Stack?5pointer?5corruption@ 00405f44     MSVCRT:userapi.obj
 0002:00000f60       ??_C@_0CK@FEGOIOPB@Cast?5to?5smaller?5type?5causing?5lo@ 00405f60     MSVCRT:userapi.obj
 0002:00000f8c       ??_C@_0BI@CIGMDCBH@Stack?5memory?5corruption@ 00405f8c     MSVCRT:userapi.obj
 0002:00000fa4       ??_C@_0CK@CNLNOEPB@Local?5variable?5used?5before?5init@ 00405fa4     MSVCRT:userapi.obj
 0002:00000fd0       ??_C@_0BP@OGBCLIBO@Stack?5around?5_alloca?5corrupted@ 00405fd0     MSVCRT:userapi.obj
 0002:00000ff4       ??_7exception@std@@6B@     00405ff4     MSVCRT:throw_bad_alloc.obj
 0002:00000ffc       ??_C@_0BC@EOODALEL@Unknown?5exception@ 00405ffc     MSVCRT:throw_bad_alloc.obj
 0002:00001014       ??_7bad_alloc@std@@6B@     00406014     MSVCRT:throw_bad_alloc.obj
 0002:0000101c       ??_C@_0P@GHFPNOJB@bad?5allocation@ 0040601c     MSVCRT:throw_bad_alloc.obj
 0002:00001030       ??_7bad_array_new_length@std@@6B@ 00406030     MSVCRT:throw_bad_alloc.obj
 0002:00001038       ??_C@_0BF@KINCDENJ@bad?5array?5new?5length@ 00406038     MSVCRT:throw_bad_alloc.obj
 0002:00001078       ??_C@_1EI@MLPKHBGE@?$AAa?$AAp?$AAi?$AA?9?$AAm?$AAs?$AA?9?$AAw?$AAi?$AAn?$AA?9?$AAc?$AAo?$AAr?$AAe@ 00406078     MSVCRT:pdblkup.obj
 0002:000010c0       ??_C@_1BK@JHLNAEJL@?$AAa?$AAd?$AAv?$AAa?$AAp?$AAi?$AA3?$AA2?$AA?4?$AAd?$AAl?$AAl@ 004060c0     MSVCRT:pdblkup.obj
 0002:000010dc       ??_C@_0O@COHOBMLB@RegOpenKeyExW@ 004060dc     MSVCRT:pdblkup.obj
 0002:000010ec       ??_C@_0BB@GLNAEDBD@RegQueryValueExW@ 004060ec     MSVCRT:pdblkup.obj
 0002:00001100       ??_C@_0M@HLOHPNFA@RegCloseKey@ 00406100     MSVCRT:pdblkup.obj
 0002:00001110       ??_C@_1HE@EBEAGLFB@?$AAS?$AAO?$AAF?$AAT?$AAW?$AAA?$AAR?$AAE?$AA?2?$AAW?$AAo?$AAw?$AA6?$AA4?$AA3@ 00406110     MSVCRT:pdblkup.obj
 0002:00001184       ??_C@_1BG@EABPBLLF@?$AAP?$AAr?$AAo?$AAd?$AAu?$AAc?$AAt?$AAD?$AAi?$AAr@ 00406184     MSVCRT:pdblkup.obj
 0002:0000119c       ??_C@_0BB@KCIACLNC@PDBOpenValidate5@ 0040619c     MSVCRT:pdblkup.obj
 0002:000011b0       ??_C@_01KDCPPGHE@r@        004061b0     MSVCRT:pdblkup.obj
 0002:000011b8       ??_7type_info@@6B@         004061b8     MSVCRT:std_type_info_static.obj
 0002:00001230       __load_config_used         00406230     MSVCRT:loadcfg.obj
 0002:000012d0       ??_R4exception@std@@6B@    004062d0     MSVCRT:throw_bad_alloc.obj
 0002:000012e4       ??_R3exception@std@@8      004062e4     MSVCRT:throw_bad_alloc.obj
 0002:000012f4       ??_R2exception@std@@8      004062f4     MSVCRT:throw_bad_alloc.obj
 0002:000012fc       ??_R1A@?0A@EA@exception@std@@8 004062fc     MSVCRT:throw_bad_alloc.obj
 0002:00001318       ??_R4bad_alloc@std@@6B@    00406318     MSVCRT:throw_bad_alloc.obj
 0002:0000132c       ??_R3bad_alloc@std@@8      0040632c     MSVCRT:throw_bad_alloc.obj
 0002:0000133c       ??_R2bad_alloc@std@@8      0040633c     MSVCRT:throw_bad_alloc.obj
 0002:00001348       ??_R1A@?0A@EA@bad_alloc@std@@8 00406348     MSVCRT:throw_bad_alloc.obj
 0002:00001364       ??_R4bad_array_new_length@std@@6B@ 00406364     MSVCRT:throw_bad_alloc.obj
 0002:00001378       ??_R3bad_array_new_length@std@@8 00406378     MSVCRT:throw_bad_alloc.obj
 0002:00001388       ??_R2bad_array_new_length@std@@8 00406388     MSVCRT:throw_bad_alloc.obj
 0002:00001398       ??_R1A@?0A@EA@bad_array_new_length@std@@8 00406398     MSVCRT:throw_bad_alloc.obj
 0002:000013b4       ??_R4type_info@@6B@        004063b4     MSVCRT:std_type_info_static.obj
 0002:000013c8       ??_R3type_info@@8          004063c8     MSVCRT:std_type_info_static.obj
 0002:000013d8       ??_R2type_info@@8          004063d8     MSVCRT:std_type_info_static.obj
 0002:000013e0       ??_R1A@?0A@EA@type_info@@8 004063e0     MSVCRT:std_type_info_static.obj
 0002:00001400       ___safe_se_handler_table   00406400     <linker-defined>
 0002:000016dc       ___rtc_iaa                 004066dc     MSVCRT:initsect.obj
 0002:000016e0       ___rtc_izz                 004066e0     MSVCRT:initsect.obj
 0002:000016e4       ___rtc_taa                 004066e4     MSVCRT:initsect.obj
 0002:000016e8       ___rtc_tzz                 004066e8     MSVCRT:initsect.obj
 0002:0000174c       __TI2?AVbad_alloc@std@@    0040674c     MSVCRT:throw_bad_alloc.obj
 0002:0000175c       __CTA2?AVbad_alloc@std@@   0040675c     MSVCRT:throw_bad_alloc.obj
 0002:00001768       __CT??_R0?AVbad_alloc@std@@@8??0bad_alloc@std@@QAE@ABV01@@Z12 00406768     MSVCRT:throw_bad_alloc.obj
 0002:00001784       __CT??_R0?AVexception@std@@@8??0exception@std@@QAE@ABV01@@Z12 00406784     MSVCRT:throw_bad_alloc.obj
 0002:000017a0       __TI3?AVbad_array_new_length@std@@ 004067a0     MSVCRT:throw_bad_alloc.obj
 0002:000017b0       __CTA3?AVbad_array_new_length@std@@ 004067b0     MSVCRT:throw_bad_alloc.obj
 0002:000017c0       __CT??_R0?AVbad_array_new_length@std@@@8??0bad_array_new_length@std@@QAE@ABV01@@Z12 004067c0     MSVCRT:throw_bad_alloc.obj
 0002:000017dc       __IMPORT_DESCRIPTOR_ADVAPI32 004067dc     advapi32:ADVAPI32.dll
 0002:000017f0       __IMPORT_DESCRIPTOR_VERSION 004067f0     version:VERSION.dll
 0002:00001804       __IMPORT_DESCRIPTOR_USER32 00406804     user32:USER32.dll
 0002:00001818       __IMPORT_DESCRIPTOR_KERNEL32 00406818     kernel32:KERNEL32.dll
 0002:0000182c       __IMPORT_DESCRIPTOR_VCRUNTIME140 0040682c     vcruntime:VCRUNTIME140.dll
 0002:00001840       __IMPORT_DESCRIPTOR_api-ms-win-crt-stdio-l1-1-0 00406840     ucrt:api-ms-win-crt-stdio-l1-1-0.dll
 0002:00001854       __IMPORT_DESCRIPTOR_api-ms-win-crt-runtime-l1-1-0 00406854     ucrt:api-ms-win-crt-runtime-l1-1-0.dll
 0002:00001868       __IMPORT_DESCRIPTOR_api-ms-win-crt-filesystem-l1-1-0 00406868     ucrt:api-ms-win-crt-filesystem-l1-1-0.dll
 0002:0000187c       __IMPORT_DESCRIPTOR_api-ms-win-crt-string-l1-1-0 0040687c     ucrt:api-ms-win-crt-string-l1-1-0.dll
 0002:00001890       __IMPORT_DESCRIPTOR_api-ms-win-crt-heap-l1-1-0 00406890     ucrt:api-ms-win-crt-heap-l1-1-0.dll
 0002:000018a4       __IMPORT_DESCRIPTOR_api-ms-win-crt-environment-l1-1-0 004068a4     ucrt:api-ms-win-crt-environment-l1-1-0.dll
 0002:000018b8       __IMPORT_DESCRIPTOR_api-ms-win-crt-math-l1-1-0 004068b8     ucrt:api-ms-win-crt-math-l1-1-0.dll
 0002:000018cc       __IMPORT_DESCRIPTOR_api-ms-win-crt-locale-l1-1-0 004068cc     ucrt:api-ms-win-crt-locale-l1-1-0.dll
 0002:000018e0       __NULL_IMPORT_DESCRIPTOR   004068e0     advapi32:ADVAPI32.dll
 0003:00000010       ___security_cookie_complement 00408010     MSVCRT:gs_cookie.obj
 0003:00000014       ___security_cookie         00408014     MSVCRT:gs_cookie.obj
 0003:00000018       ?_RTC_ErrorLevels@@3PAHA   00408018     MSVCRT:error.obj
 0003:0000002c       ___scrt_native_dllmain_reason 0040802c     MSVCRT:utility.obj
 0003:00000030       ___scrt_default_matherr    00408030     MSVCRT:matherr.obj
 0003:00000040       ___isa_enabled             00408040     MSVCRT:cpu_disp.obj
 0003:00000044       ___scrt_ucrt_dll_is_in_use 00408044     MSVCRT:ucrt_stubs.obj
 0003:00000048       ??_R0?AVbad_alloc@std@@@8  00408048     MSVCRT:throw_bad_alloc.obj
 0003:00000064       ??_R0?AVexception@std@@@8  00408064     MSVCRT:throw_bad_alloc.obj
 0003:00000080       ??_R0?AVbad_array_new_length@std@@@8 00408080     MSVCRT:throw_bad_alloc.obj
 0003:000000a8       ??_R0?AVtype_info@@@8      004080a8     MSVCRT:std_type_info_static.obj
 0003:000000c0       ?origFile@@3PAU_iobuf@@A   004080c0     jabswitch.obj
 0003:000000c4       ?tempFile@@3PAU_iobuf@@A   004080c4     jabswitch.obj
 0003:000000c8       ?_OptionsStorage@?1??__local_stdio_printf_options@@9@4_KA 004080c8     jabswitch.obj
 0003:000003fc       ___scrt_current_native_startup_state 004083fc     MSVCRT:utility.obj
 0003:00000400       ___scrt_native_startup_lock 00408400     MSVCRT:utility.obj
 0003:00000420       ?__type_info_root_node@@3U__type_info_node@@A 00408420     MSVCRT:tncleanup.obj
 0003:00000428       ?_OptionsStorage@?1??__local_stdio_scanf_options@@9@4_KA 00408428     MSVCRT:default_local_stdio_options.obj
 0003:00000430       ___scrt_debugger_hook_flag 00408430     MSVCRT:utility_desktop.obj
 0003:0000043c       ___isa_available           0040843c     MSVCRT:cpu_disp.obj
 0003:00000440       ___favor                   00408440     MSVCRT:cpu_disp.obj
 0003:00000444       ___dyn_tls_dtor_callback   00408444     <common>
 0003:00000448       ___dyn_tls_init_callback   00408448     <common>

 entry point at        0001:0000245a

 Static symbols

 0000:ffff5000       .debug$S                   00400000     advapi32:ADVAPI32.dll
 0000:ffff5000       .debug$S                   00400000     advapi32:ADVAPI32.dll
 0000:ffff5000       .debug$S                   00400000     advapi32:ADVAPI32.dll
 0000:ffff5000       .debug$S                   00400000     advapi32:ADVAPI32.dll
 0000:ffff5000       .debug$S                   00400000     version:VERSION.dll
 0000:ffff5000       .debug$S                   00400000     version:VERSION.dll
 0000:ffff5000       .debug$S                   00400000     version:VERSION.dll
 0000:ffff5000       .debug$S                   00400000     user32:USER32.dll
 0000:ffff5000       .debug$S                   00400000     kernel32:KERNEL32.dll
 0000:ffff5000       .debug$S                   00400000     kernel32:KERNEL32.dll
 0000:ffff5000       .debug$S                   00400000     kernel32:KERNEL32.dll
 0000:ffff5000       .debug$S                   00400000     ucrt:api-ms-win-crt-runtime-l1-1-0.dll
 0000:ffff5000       .debug$S                   00400000     ucrt:api-ms-win-crt-runtime-l1-1-0.dll
 0000:ffff5000       .debug$S                   00400000     ucrt:api-ms-win-crt-runtime-l1-1-0.dll
 0000:ffff5000       .debug$S                   00400000     ucrt:api-ms-win-crt-runtime-l1-1-0.dll
 0000:ffff5000       .debug$S                   00400000     ucrt:api-ms-win-crt-runtime-l1-1-0.dll
 0000:ffff5000       .debug$S                   00400000     ucrt:api-ms-win-crt-runtime-l1-1-0.dll
 0000:ffff5000       .debug$S                   00400000     ucrt:api-ms-win-crt-runtime-l1-1-0.dll
 0000:ffff5000       .debug$S                   00400000     ucrt:api-ms-win-crt-runtime-l1-1-0.dll
 0000:ffff5000       .debug$S                   00400000     ucrt:api-ms-win-crt-heap-l1-1-0.dll
 0000:ffff5000       .debug$S                   00400000     ucrt:api-ms-win-crt-heap-l1-1-0.dll
 0000:ffff5000       .debug$S                   00400000     ucrt:api-ms-win-crt-stdio-l1-1-0.dll
 0000:ffff5000       .debug$S                   00400000     ucrt:api-ms-win-crt-heap-l1-1-0.dll
 0000:ffff5000       .debug$S                   00400000     ucrt:api-ms-win-crt-locale-l1-1-0.dll
 0000:ffff5000       .debug$S                   00400000     ucrt:api-ms-win-crt-runtime-l1-1-0.dll
 0000:ffff5000       .debug$S                   00400000     ucrt:api-ms-win-crt-runtime-l1-1-0.dll
 0000:ffff5000       .debug$S                   00400000     ucrt:api-ms-win-crt-runtime-l1-1-0.dll
 0000:ffff5000       .debug$S                   00400000     ucrt:api-ms-win-crt-runtime-l1-1-0.dll
 0000:ffff5000       .debug$S                   00400000     ucrt:api-ms-win-crt-runtime-l1-1-0.dll
 0000:ffff5000       .debug$S                   00400000     ucrt:api-ms-win-crt-stdio-l1-1-0.dll
 0000:ffff5000       .debug$S                   00400000     ucrt:api-ms-win-crt-runtime-l1-1-0.dll
 0000:ffff5000       .debug$S                   00400000     ucrt:api-ms-win-crt-runtime-l1-1-0.dll
 0000:ffff5000       .debug$S                   00400000     ucrt:api-ms-win-crt-runtime-l1-1-0.dll
 0000:ffff5000       .debug$S                   00400000     ucrt:api-ms-win-crt-runtime-l1-1-0.dll
 0000:ffff5000       .debug$S                   00400000     ucrt:api-ms-win-crt-runtime-l1-1-0.dll
 0000:ffff5000       .debug$S                   00400000     ucrt:api-ms-win-crt-runtime-l1-1-0.dll
 0000:ffff5000       .debug$S                   00400000     ucrt:api-ms-win-crt-math-l1-1-0.dll
 0000:ffff5000       .debug$S                   00400000     ucrt:api-ms-win-crt-runtime-l1-1-0.dll
 0000:ffff5000       .debug$S                   00400000     ucrt:api-ms-win-crt-runtime-l1-1-0.dll
 0000:ffff5000       .debug$S                   00400000     ucrt:api-ms-win-crt-environment-l1-1-0.dll
 0000:ffff5000       .debug$S                   00400000     ucrt:api-ms-win-crt-runtime-l1-1-0.dll
 0000:ffff5000       .debug$S                   00400000     ucrt:api-ms-win-crt-heap-l1-1-0.dll
 0000:ffff5000       .debug$S                   00400000     ucrt:api-ms-win-crt-string-l1-1-0.dll
 0000:ffff5000       .debug$S                   00400000     ucrt:api-ms-win-crt-string-l1-1-0.dll
 0000:ffff5000       .debug$S                   00400000     ucrt:api-ms-win-crt-string-l1-1-0.dll
 0000:ffff5000       .debug$S                   00400000     ucrt:api-ms-win-crt-string-l1-1-0.dll
 0000:ffff5000       .debug$S                   00400000     ucrt:api-ms-win-crt-string-l1-1-0.dll
 0000:ffff5000       .debug$S                   00400000     ucrt:api-ms-win-crt-string-l1-1-0.dll
 0000:ffff5000       .debug$S                   00400000     ucrt:api-ms-win-crt-string-l1-1-0.dll
 0000:ffff5000       .debug$S                   00400000     ucrt:api-ms-win-crt-string-l1-1-0.dll
 0000:ffff5000       .debug$S                   00400000     ucrt:api-ms-win-crt-string-l1-1-0.dll
 0000:ffff5000       .debug$S                   00400000     ucrt:api-ms-win-crt-runtime-l1-1-0.dll
 0000:ffff5000       .debug$S                   00400000     ucrt:api-ms-win-crt-stdio-l1-1-0.dll
 0000:ffff5000       .debug$S                   00400000     ucrt:api-ms-win-crt-stdio-l1-1-0.dll
 0000:ffff5000       .debug$S                   00400000     ucrt:api-ms-win-crt-filesystem-l1-1-0.dll
 0000:ffff5000       .debug$S                   00400000     ucrt:api-ms-win-crt-filesystem-l1-1-0.dll
 0000:ffff5000       .debug$S                   00400000     ucrt:api-ms-win-crt-runtime-l1-1-0.dll
 0000:ffff5000       .debug$S                   00400000     ucrt:api-ms-win-crt-stdio-l1-1-0.dll
 0000:ffff5000       .debug$S                   00400000     ucrt:api-ms-win-crt-stdio-l1-1-0.dll
 0000:ffff5000       .debug$S                   00400000     ucrt:api-ms-win-crt-stdio-l1-1-0.dll
 0000:ffff5000       .debug$S                   00400000     ucrt:api-ms-win-crt-stdio-l1-1-0.dll
 0000:ffff5000       .debug$S                   00400000     ucrt:api-ms-win-crt-stdio-l1-1-0.dll
 0000:ffff5000       .debug$S                   00400000     ucrt:api-ms-win-crt-stdio-l1-1-0.dll
 0000:ffff5000       .debug$S                   00400000     kernel32:KERNEL32.dll
 0000:ffff5000       .debug$S                   00400000     vcruntime:VCRUNTIME140.dll
 0000:ffff5000       .debug$S                   00400000     vcruntime:VCRUNTIME140.dll
 0000:ffff5000       .debug$S                   00400000     vcruntime:VCRUNTIME140.dll
 0000:ffff5000       .debug$S                   00400000     vcruntime:VCRUNTIME140.dll
 0000:ffff5000       .debug$S                   00400000     vcruntime:VCRUNTIME140.dll
 0000:ffff5000       .debug$S                   00400000     vcruntime:VCRUNTIME140.dll
 0000:ffff5000       .debug$S                   00400000     vcruntime:VCRUNTIME140.dll
 0000:ffff5000       .debug$S                   00400000     vcruntime:VCRUNTIME140.dll
 0000:ffff5000       .debug$S                   00400000     vcruntime:VCRUNTIME140.dll
 0000:ffff5000       .debug$S                   00400000     vcruntime:VCRUNTIME140.dll
 0000:ffff5000       .debug$S                   00400000     kernel32:KERNEL32.dll
 0000:ffff5000       .debug$S                   00400000     kernel32:KERNEL32.dll
 0000:ffff5000       .debug$S                   00400000     kernel32:KERNEL32.dll
 0000:ffff5000       .debug$S                   00400000     kernel32:KERNEL32.dll
 0000:ffff5000       .debug$S                   00400000     kernel32:KERNEL32.dll
 0000:ffff5000       .debug$S                   00400000     kernel32:KERNEL32.dll
 0000:ffff5000       .debug$S                   00400000     kernel32:KERNEL32.dll
 0000:ffff5000       .debug$S                   00400000     kernel32:KERNEL32.dll
 0000:ffff5000       .debug$S                   00400000     kernel32:KERNEL32.dll
 0000:ffff5000       .debug$S                   00400000     kernel32:KERNEL32.dll
 0000:ffff5000       .debug$S                   00400000     kernel32:KERNEL32.dll
 0000:ffff5000       .debug$S                   00400000     kernel32:KERNEL32.dll
 0000:ffff5000       .debug$S                   00400000     kernel32:KERNEL32.dll
 0000:ffff5000       .debug$S                   00400000     kernel32:KERNEL32.dll
 0000:ffff5000       .debug$S                   00400000     kernel32:KERNEL32.dll
 0000:ffff5000       .debug$S                   00400000     kernel32:KERNEL32.dll
 0000:ffff5000       .debug$S                   00400000     kernel32:KERNEL32.dll
 0000:ffff5000       .debug$S                   00400000     kernel32:KERNEL32.dll
 0000:ffff5000       .debug$S                   00400000     kernel32:KERNEL32.dll
 0000:ffff5000       .debug$S                   00400000     kernel32:KERNEL32.dll
 0000:ffff5000       .debug$S                   00400000     kernel32:KERNEL32.dll
 0000:ffff5000       .debug$S                   00400000     kernel32:KERNEL32.dll
 0001:000000b0       $LN6                       004010b0     jabswitch.obj
 0001:000000b8       $LN5                       004010b8     jabswitch.obj
 0001:000000c4       $LN4                       004010c4     jabswitch.obj
 0001:0000052c       $LN31                      0040152c     jabswitch.obj
 0001:00000534       $LN30                      00401534     jabswitch.obj
 0001:0000057c       $LN29                      0040157c     jabswitch.obj
 0001:00000584       $LN28                      00401584     jabswitch.obj
 0001:0000058c       $LN27                      0040158c     jabswitch.obj
 0001:00000594       $LN26                      00401594     jabswitch.obj
 0001:0000059c       $LN25                      0040159c     jabswitch.obj
 0001:000005a8       $LN24                      004015a8     jabswitch.obj
 0001:00000800       $LN19                      00401800     jabswitch.obj
 0001:00000808       $LN18                      00401808     jabswitch.obj
 0001:00000838       $LN17                      00401838     jabswitch.obj
 0001:00000840       $LN16                      00401840     jabswitch.obj
 0001:00000848       $LN15                      00401848     jabswitch.obj
 0001:00000854       $LN14                      00401854     jabswitch.obj
 0001:00000d34       $LN29                      00401d34     jabswitch.obj
 0001:00000d3c       $LN28                      00401d3c     jabswitch.obj
 0001:00000d90       $LN27                      00401d90     jabswitch.obj
 0001:00000d94       $LN26                      00401d94     jabswitch.obj
 0001:00000d9f       $LN25                      00401d9f     jabswitch.obj
 0001:00000daa       $LN24                      00401daa     jabswitch.obj
 0001:00000dae       $LN23                      00401dae     jabswitch.obj
 0001:00000dba       $LN22                      00401dba     jabswitch.obj
 0001:00000dc3       $LN21                      00401dc3     jabswitch.obj
 0001:0000109c       $LN14                      0040209c     jabswitch.obj
 0001:000010a4       $LN13                      004020a4     jabswitch.obj
 0001:000010ec       $LN12                      004020ec     jabswitch.obj
 0001:000010f9       $LN11                      004020f9     jabswitch.obj
 0001:00001107       $LN10                      00402107     jabswitch.obj
 0001:0000110d       $LN9                       0040210d     jabswitch.obj
 0001:0000111a       $LN8                       0040211a     jabswitch.obj
 0001:00001121       $LN7                       00402121     jabswitch.obj
 0001:000013b4       $LN16                      004023b4     jabswitch.obj
 0001:000013bc       $LN15                      004023bc     jabswitch.obj
 0001:000013ec       $LN14                      004023ec     jabswitch.obj
 0001:000013f7       $LN13                      004023f7     jabswitch.obj
 0001:00001402       $LN12                      00402402     jabswitch.obj
 0001:0000140b       $LN11                      0040240b     jabswitch.obj
 0001:000017d4       $LN23                      004027d4     jabswitch.obj
 0001:000017dc       $LN22                      004027dc     jabswitch.obj
 0001:00001824       $LN21                      00402824     jabswitch.obj
 0001:0000182e       $LN20                      0040282e     jabswitch.obj
 0001:0000183b       $LN19                      0040283b     jabswitch.obj
 0001:00001846       $LN18                      00402846     jabswitch.obj
 0001:00001851       $LN17                      00402851     jabswitch.obj
 0001:0000185a       $LN16                      0040285a     jabswitch.obj
 0001:00001940       $LN7                       00402940     jabswitch.obj
 0001:00001948       $LN6                       00402948     jabswitch.obj
 0001:00001960       $LN5                       00402960     jabswitch.obj
 0001:0000196c       $LN4                       0040296c     jabswitch.obj
 0001:00002213       ?pre_c_initialization@@YAHXZ 00403213 f   MSVCRT:exe_main.obj
 0001:000022be       ?post_pgo_initialization@@YAHXZ 004032be f   MSVCRT:exe_main.obj
 0001:000022c6       ?pre_cpp_initialization@@YAXXZ 004032c6 f   MSVCRT:exe_main.obj
 0001:000022d8       ?__scrt_common_main_seh@@YAHXZ 004032d8 f   MSVCRT:exe_main.obj
 0001:00002576       ?failwithmessage@@YAXPAXHHPBD@Z 00403576 f   MSVCRT:error.obj
 0001:000027dd       ?notify_debugger@@YAXABUtagEXCEPTION_VISUALCPP_DEBUG_INFO@@@Z 004037dd f   MSVCRT:error.obj
 0001:0000283a       ?find_pe_section@@YAPAU_IMAGE_SECTION_HEADER@@QAEI@Z 0040383a f   MSVCRT:utility.obj
 0001:00002ab7       ___get_entropy             00403ab7 f   MSVCRT:gs_support.obj
 0001:00002de0       $$000000                   00403de0     MSVCRT:sehprolg4.obj
 0001:00002f77       ?GetPdbDllFromInstallPath@@YAPAUHINSTANCE__@@XZ 00403f77 f   MSVCRT:pdblkup.obj
 0002:000001a8       ?pre_cpp_initializer@@3P6AXXZA 004051a8     MSVCRT:exe_main.obj
 0002:000001b4       ?pre_c_initializer@@3P6AHXZA 004051b4     MSVCRT:exe_main.obj
 0002:000001b8       ?post_pgo_initializer@@3P6AHXZA 004051b8     MSVCRT:exe_main.obj
 0002:000001d0       $SG45722                   004051d0     jabswitch.obj
 0002:00000248       $SG45724                   00405248     jabswitch.obj
 0002:000002d0       $SG45726                   004052d0     jabswitch.obj
 0002:000002ec       $SG45728                   004052ec     jabswitch.obj
 0002:0000031c       $SG45756                   0040531c     jabswitch.obj
 0002:00000320       $SG45757                   00405320     jabswitch.obj
 0002:00000360       $SG45758                   00405360     jabswitch.obj
 0002:00000380       $SG45762                   00405380     jabswitch.obj
 0002:000003c4       $SG45767                   004053c4     jabswitch.obj
 0002:000003dc       $SG45768                   004053dc     jabswitch.obj
 0002:000003e0       $SG45773                   004053e0     jabswitch.obj
 0002:00000400       $SG45778                   00405400     jabswitch.obj
 0002:0000041c       $SG45779                   0040541c     jabswitch.obj
 0002:00000420       $SG45802                   00405420     jabswitch.obj
 0002:00000438       $SG45803                   00405438     jabswitch.obj
 0002:0000043c       $SG45806                   0040543c     jabswitch.obj
 0002:00000440       $SG45809                   00405440     jabswitch.obj
 0002:0000045c       $SG45810                   0040545c     jabswitch.obj
 0002:00000460       $SG45813                   00405460     jabswitch.obj
 0002:00000464       $SG45837                   00405464     jabswitch.obj
 0002:00000470       $SG45839                   00405470     jabswitch.obj
 0002:00000490       $SG45840                   00405490     jabswitch.obj
 0002:00000498       $SG45841                   00405498     jabswitch.obj
 0002:000004b4       $SG45842                   004054b4     jabswitch.obj
 0002:000004d0       $SG45845                   004054d0     jabswitch.obj
 0002:00000504       $SG45846                   00405504     jabswitch.obj
 0002:00000530       $SG45847                   00405530     jabswitch.obj
 0002:00000534       $SG45852                   00405534     jabswitch.obj
 0002:00000538       $SG45855                   00405538     jabswitch.obj
 0002:00000554       $SG45856                   00405554     jabswitch.obj
 0002:0000055c       $SG45858                   0040555c     jabswitch.obj
 0002:0000057c       $SG45859                   0040557c     jabswitch.obj
 0002:00000580       $SG45857                   00405580     jabswitch.obj
 0002:000005c0       $SG45861                   004055c0     jabswitch.obj
 0002:000005e0       $SG45862                   004055e0     jabswitch.obj
 0002:000005e8       $SG45866                   004055e8     jabswitch.obj
 0002:00000604       $SG45867                   00405604     jabswitch.obj
 0002:0000060c       $SG45869                   0040560c     jabswitch.obj
 0002:00000628       $SG45870                   00405628     jabswitch.obj
 0002:00000630       $SG45873                   00405630     jabswitch.obj
 0002:00000664       $SG45874                   00405664     jabswitch.obj
 0002:00000674       $SG45875                   00405674     jabswitch.obj
 0002:000006b0       $SG45876                   004056b0     jabswitch.obj
 0002:000006c0       $SG45877                   004056c0     jabswitch.obj
 0002:000006f4       $SG45878                   004056f4     jabswitch.obj
 0002:00000728       $SG45879                   00405728     jabswitch.obj
 0002:0000074c       $SG45880                   0040574c     jabswitch.obj
 0002:0000077c       $SG45881                   0040577c     jabswitch.obj
 0002:00000784       $SG45882                   00405784     jabswitch.obj
 0002:000007bc       $SG45883                   004057bc     jabswitch.obj
 0002:000007f4       $SG45884                   004057f4     jabswitch.obj
 0002:00000830       $SG45885                   00405830     jabswitch.obj
 0002:0000086c       $SG45886                   0040586c     jabswitch.obj
 0002:000008a8       $SG45887                   004058a8     jabswitch.obj
 0002:000008e4       $SG45888                   004058e4     jabswitch.obj
 0002:0000090c       $SG45914                   0040590c     jabswitch.obj
 0002:00000934       $SG45916                   00405934     jabswitch.obj
 0002:00000958       $SG45918                   00405958     jabswitch.obj
 0002:00000978       $SG45920                   00405978     jabswitch.obj
 0002:0000097c       $SG45921                   0040597c     jabswitch.obj
 0002:0000099c       $SG45922                   0040599c     jabswitch.obj
 0002:000009b0       $SG45923                   004059b0     jabswitch.obj
 0002:000009bc       $SG45924                   004059bc     jabswitch.obj
 0002:000009f4       $SG45955                   004059f4     jabswitch.obj
 0002:00000a00       $SG45992                   00405a00     jabswitch.obj
 0002:00000a04       $SG45993                   00405a04     jabswitch.obj
 0002:00000a08       $SG45997                   00405a08     jabswitch.obj
 0002:00000a0c       $SG45998                   00405a0c     jabswitch.obj
 0002:00000a10       $SG46011                   00405a10     jabswitch.obj
 0002:00000a1c       $SG46024                   00405a1c     jabswitch.obj
 0002:00000a20       $SG46025                   00405a20     jabswitch.obj
 0002:00000a24       $SG46029                   00405a24     jabswitch.obj
 0002:00000a30       $SG46030                   00405a30     jabswitch.obj
 0002:00000a3c       $SG46034                   00405a3c     jabswitch.obj
 0002:00000a44       $SG46035                   00405a44     jabswitch.obj
 0002:00000a4c       $SG46040                   00405a4c     jabswitch.obj
 0002:00000a58       $SG46041                   00405a58     jabswitch.obj
 0002:00000a64       $SG46049                   00405a64     jabswitch.obj
 0002:00000a7c       $SG46050                   00405a7c     jabswitch.obj
 0002:00000a98       $SG46052                   00405a98     jabswitch.obj
 0002:00000aa0       $SG46053                   00405aa0     jabswitch.obj
 0002:00000aa8       $SG46056                   00405aa8     jabswitch.obj
 0002:00000ab4       $SG46057                   00405ab4     jabswitch.obj
 0002:00000ac0       _GS_ExceptionPointers      00405ac0     MSVCRT:gs_report.obj
 0002:00000ac8       ?_RTC_ErrorMessages@@3QBQBDB 00405ac8     MSVCRT:error.obj
 0002:00000ae0       ?_RTC_NoFalsePositives@@3QBHB 00405ae0     MSVCRT:error.obj
 0002:00000af8       ?stack_premsg@@3QBDB       00405af8     MSVCRT:error.obj
 0002:00000b14       ?stack_postmsg@@3QBDB      00405b14     MSVCRT:error.obj
 0002:00000b28       ?uninit_premsg@@3QBDB      00405b28     MSVCRT:error.obj
 0002:00000b38       ?uninit_postmsg@@3QBDB     00405b38     MSVCRT:error.obj
 0002:00000f30       ?_RTC_errlist@@3QBQBDB     00405f30     MSVCRT:userapi.obj
 0002:00001050       ?mspdbName@@3QB_WB         00406050     MSVCRT:pdblkup.obj
 0002:000016f0       __sehtable$?__scrt_common_main_seh@@YAHXZ 004066f0     MSVCRT:exe_main.obj
 0002:00001710       __sehtable$?notify_debugger@@YAXABUtagEXCEPTION_VISUALCPP_DEBUG_INFO@@@Z 00406710     MSVCRT:error.obj
 0002:00001730       __sehtable$___scrt_is_nonwritable_in_current_image 00406730     MSVCRT:utility.obj
 0002:00001ad8       .idata$6                   00406ad8     advapi32:ADVAPI32.dll
 0002:00001b28       .idata$6                   00406b28     version:VERSION.dll
 0002:00001b40       .idata$6                   00406b40     user32:USER32.dll
 0002:00001d4e       .idata$6                   00406d4e     kernel32:KERNEL32.dll
 0002:00001e10       .idata$6                   00406e10     vcruntime:VCRUNTIME140.dll
 0002:00002114       .idata$6                   00407114     ucrt:api-ms-win-crt-stdio-l1-1-0.dll
 0002:00002134       .idata$6                   00407134     ucrt:api-ms-win-crt-runtime-l1-1-0.dll
 0002:00002156       .idata$6                   00407156     ucrt:api-ms-win-crt-filesystem-l1-1-0.dll
 0002:0000217c       .idata$6                   0040717c     ucrt:api-ms-win-crt-string-l1-1-0.dll
 0002:0000219e       .idata$6                   0040719e     ucrt:api-ms-win-crt-heap-l1-1-0.dll
 0002:000021be       .idata$6                   004071be     ucrt:api-ms-win-crt-environment-l1-1-0.dll
 0002:000021e4       .idata$6                   004071e4     ucrt:api-ms-win-crt-math-l1-1-0.dll
 0002:00002204       .idata$6                   00407204     ucrt:api-ms-win-crt-locale-l1-1-0.dll
 0003:00000000       ?ACCESSIBILITY_USER_KEY@@3PB_WB 00408000     jabswitch.obj
 0003:00000004       ?ACCESSIBILITY_SYSTEM_KEY@@3PB_WB 00408004     jabswitch.obj
 0003:00000008       ?ACCESSIBILITY_CONFIG@@3PB_WB 00408008     jabswitch.obj
 0003:0000000c       ?STR_ACCESSBRIDGE@@3PB_WB  0040800c     jabswitch.obj
 0003:000000d0       ?isXPFlag@?1??isXP@@YA_NXZ@4_NA 004080d0     jabswitch.obj
 0003:000000d8       _GS_ExceptionRecord        004080d8     MSVCRT:gs_report.obj
 0003:00000128       _GS_ContextRecord          00408128     MSVCRT:gs_report.obj
 0003:000003f4       ?_RTC_ErrorReportFunc@@3P6AHHPBDH00ZZA 004083f4     MSVCRT:userapi.obj
 0003:000003f8       ?_RTC_ErrorReportFuncW@@3P6AHHPB_WH00ZZA 004083f8     MSVCRT:userapi.obj
 0003:00000404       ?is_initialized_as_dll@@3_NA 00408404     MSVCRT:utility.obj
 0003:00000405       ?module_local_atexit_table_initialized@@3_NA 00408405     MSVCRT:utility.obj
 0003:00000408       ?module_local_atexit_table@@3U_onexit_table_t@@A 00408408     MSVCRT:utility.obj
 0003:00000414       ?module_local_at_quick_exit_table@@3U_onexit_table_t@@A 00408414     MSVCRT:utility.obj
 0003:00000434       ?mspdb@@3PAUHINSTANCE__@@A 00408434     MSVCRT:pdblkup.obj
 0003:00000438       ?alreadyTried@?1??GetPdbDll@@YAPAUHINSTANCE__@@XZ@4_NA 00408438     MSVCRT:pdblkup.obj
 0003:00000439       ?PDBOK@?1??_RTC_GetSrcLine@@YAHPAEPA_WKPAH1K@Z@4_NA 00408439     MSVCRT:pdblkup.obj
 0004:00000120       $R000000                   00409120     jabswitch.exe.res
 0004:00000338       $R000218                   00409338     jabswitch.exe.res
 0004:000003c8       $R0002A8                   004093c8     jabswitch.exe.res
